:020000040000FA
:020000000828CE
:04000800FC2A0900C5
:100010008316031307309F001030850000308600E0
:1000200000308700003088000030890083120313FD
:100030003130900000308E0000308F0083160313A3
:10004000E0308B0001308C000130810083120313FB
:10005000F0308400D200D300FF3085008600870096
:1000600088008900EA019A200739DA000630D800B2
:100070001E30BE002030C000FF30850087004008E1
:100080008400FF308000C00ABE0B3C286C236C2328
:100090006C234F206C23D80B38284F205A28183057
:1000A000BE002030C000400884008001C00ABE0BA2
:1000B000532808000630BF00BD01C101C201BC20A9
:1000C0004218BB20051A60285A0A0739DA00A52011
:1000D0006C236C236C235A08313EC401C500031005
:1000E000C50DC40D0310C50DC40D0310C50DC40D01
:1000F00044164F2023218A110A12A800C50A232181
:100100008A110A12A900C50A23218A110A12AA001B
:10011000C50A23218A110A12AB00C50A23218A11BC
:100120000A12AC00C50A0630BF00BD01C101C20100
:10013000BC2060280317831210308D0083168C13A7
:100140000C1483120C0803130800031783168C1871
:10015000A72883128C0010308D0083168C130C1589
:100160008B1355308D00AA308D008C148B170C1119
:10017000031383120800C10A00305A02031DC2286B
:100180002721C300000001305A02031DC928532152
:10019000C300000002305A02031DD0287521C3009D
:1001A000000003305A02031DD7289621C300000027
:1001B00004305A02031DDE28B021C30000000530C0
:1001C0005A02031DE528D321C300000006305A025D
:1001D000031DEC28EF21C300000007305A02031D65
:1001E000F3280D22C30000004308003E0319212913
:1001F000C4014308C5000310C50DC40D0310C50D8F
:10020000C40D0310C50DC40D441623218A110A1212
:10021000B800C50A23218A110A12B900C50A232190
:100220008A110A12BA00C50A23218A110A12BB00D8
:10023000C50A23218A110A12BC00C50ABD01421059
:100240000800C1015A2844088A0045088200410874
:10025000E70001308A003030670703188A0A8200FD
:1002600045344A34203465346A342034B434DA34C2
:10027000B734BC34DE34AC34AF34B8342034BA34A0
:10028000B334CB34AE34B3342034CA34C234CA3479
:10029000DE34B234C134AD34B334203420342034AD
:1002A0002034003400344108E70001308A005C301B
:1002B000670703188A0A82005434683461346E3444
:1002C0006B34203479346F34753421342134213443
:1002D0002034B134D834B634DE34C434B3342034AA
:1002E000203420342034003400344108E700013049
:1002F0008A007E30670703188A0A820048346F3408
:1003000077342034613472346534203479346F3476
:1003100075343F342034B934DE34DD34B7343F34FF
:100320002034203420342034003400344108E700E5
:1003300001308A009F30670703188A0A820053340D
:100340006F347234723479342034BD34D034CF34C5
:10035000BE34DD34203420342034203400340034E2
:100360004108E70001308A00B930670703188A0A9C
:1003700082004E346F34773420346F346E3420343E
:10038000533441344C3445342034B234D734AF3450
:10039000BC34AC34B234CF34BE34203420342034B6
:1003A0002034003400344108E70001308A00DC309A
:1003B000670703188A0A82004F34503445344E349C
:1003C0002034B234D734AF34BC34AC34B234CF344C
:1003D000BE3420342034203420340034003441082A
:1003E000E70001308A00F830670703188A0A8200A4
:1003F00043344C344F34533445342034CD34B23448
:10040000C334DD342034BC34CF34BC34C034203465
:10041000203420342034003400344108E700023016
:100420008A001630670703188A0A8200533454344E
:100430004F3450342034C234B234C434C234203443
:10044000C134AD34B034B2342034203420342034BC
:10045000003400340B11003081006B0A0739EB00C7
:1004600000306B020319512A01306B020319632A11
:1004700002306B020319752A03306B020319872AB5
:1004800004306B020319992A05306B020319AB2A59
:1004900006306B020319BD2A07306B020319CF2AFD
:1004A0000800200886002808880030088900D70046
:1004B000D70CD70CD70CD712571AD7165708850068
:1004C000803087000800210886002908880031084C
:1004D0008900D700D70CD70CD70CD712571AD716CC
:1004E00057088500403087000800220886002A0847
:1004F000880032088900D700D70CD70CD70CD71248
:10050000571AD7165708850020308700080023089F
:1005100086002B08880033088900D700D70CD70C39
:10052000D70CD712571AD7165708850010308700F6
:100530000800240886002C08880034088900D700A9
:10054000D70CD70CD70CD712571AD71657088500D7
:10055000083087000800250886002D088800350827
:100560008900D700D70CD70CD70CD712571AD7163B
:1005700057088500043087000800260886002E08EA
:10058000880036088900D700D70CD70CD70CD712B3
:10059000571AD71657088500023087000800270829
:1005A00086002F08880037088900D700D70CD70CA1
:1005B000D70CD712571AD716570885000130870075
:1005C00008000C1000308E0000308F00EF22BF0BAF
:1005D00008000630BF0042140800EA0308001E307D
:1005E000BE002030C000400A840000088403800060
:1005F000C00ABE0BF32A0800C60003088301C70027
:100600000A08CA000408CB008A110A128B1A0B1DB3
:100610000A2B2A220B1A8B1C0E2B00008B190B1C89
:10062000122B00000B1F332B831203130C088316AD
:1006300003130C0583120313CC004C1B0000CC1ACF
:100640004C1A00004C190000CC1800004C18E12294
:10065000831203130D08831603130D05831203136E
:10066000CC004C18000083014B0884004A088A0023
:1006700047088300C60E460E09000730DF00DF0B77
:100680003F2B08000930E0003D23E00B442B08001D
:100690005A30E1003D23E10B4A2B08002F30E200E5
:1006A0004223E20B502B08006230E2004223E20BAF
:1006B000562B08003130E3004823E30B5C2B080085
:1006C0006330E4004E23E40B622B08001430E40096
:1006D0004823E40B682B08006430E4004823E40B53
:1006E0006E2B0800FA30E4004823E40B742B08005A
:102000000034003400340034003400340034003430
:102010000034003400340034003400340034003420
:102020000034003400340034003400340034003410
:102030000034003400340034003400340034003400
:10221000003400345F3400340034003400340034BF
:102220000B34073400340B340734003400340034EA
:1022300014347F3414347F341434003400340034C4
:1022400024342A347F342A341234003400340034E5
:1022500023341334083464346234003400340034DA
:102260003634493455342234503400340034003488
:10227000003400340B3407340034003400340034AC
:1022800000341C342234413400340034003400342F
:102290000034413422341C3400340034003400341F
:1022A000143408343E340834143400340034003418
:1022B000083408343E340834083400340034003420
:1022C00000340034583438340034003400340034DE
:1022D0000834083408340834083400340034003436
:1022E000003460346034003400340034003400348E
:1022F0002034103408340434023400340034003400
:102300003E345134493445343E34003400340034D2
:10231000003442347F34403400340034003400341C
:10232000423461345134493446340034003400348A
:102330002134413445344B343134003400340034DA
:102340001834143412347F34103400340034003420
:1023500027344534453445343934003400340034AE
:102360003C344A3449344934303400340034003485
:102370000334013471340934073400340034003438
:102380003634493449344934363400340034003466
:1023900006344934493429341E34003400340034BE
:1023A0000034363436340034003400340034003421
:1023B00000345634363400340034003400340034F1
:1023C00000340834143422344134003400340034EE
:1023D00014341434143414341434003400340034F9
:1023E00000344134223414340834003400340034CE
:1023F00002340134513409340634003400340034DA
:102400003E3441345D3455345E340034003400349D
:102410007E340934093409347E3400340034003405
:102420007F3449344934493436340034003400347C
:102430003E344134413441342234003400340034D9
:1024400041347F34413441343E340034003400346C
:102450007F34493449344934413400340034003441
:102460007F34093409340934013400340034003431
:102470003E344134493449347A3400340034003431
:102480007F340834083408347F3400340034003496
:10249000003441347F34413400340034003400349B
:1024A0002034403441343F340134003400340034AB
:1024B0007F3408341434223441340034003400347E
:1024C0007F344034403440344034003400340034ED
:1024D0007F3402340C3402347F340034003400344E
:1024E0007F340434083410347F3400340034003432
:1024F0003E344134413441343E34003400340034FD
:102500007F3409340934093406340034003400348B
:102510003E344134513421345E34003400340034CC
:102520007F340934193429344634003400340034FB
:1025300046344934493449343134003400340034A9
:10254000013401347F340134013400340034003468
:102550003F344034403440343F340034003400349D
:102560001F342034403420341F340034003400340D
:102570003F344034383440343F3400340034003485
:1025800063341434083414346334003400340034B5
:102590000334043478340434033400340034003415
:1025A0006134513449344534433400340034003408
:1025B00000347F344134413400340034003400347A
:1025C000153416347C341634153400340034003499
:1025D0000034413441347F3400340034003400345A
:1025E000043402340134023404340034003400343E
:1025F00040344034403440344034003400340034FB
:1026000040344034403440344034003400340034EA
:102610002034543454345434783400340034003486
:102620007F34483444344434383400340034003483
:1026300038344434443444342034003400340034D6
:1026400038344434443448347F3400340034003463
:10265000383454345434543408340034003400349E
:1026600004347E340534053401340034003400343D
:1026700008345434543454343C340034003400347A
:102680007F340834043404347834003400340034A3
:10269000003408347D3440340034003400340034D5
:1026A0002034403444343D340034003400340034A9
:1026B00000347F341034283444340034003400347F
:1026C00000343F34403440340034003400340034AB
:1026D0007C34043418340434783400340034003446
:1026E0007C34083404340434783400340034003446
:1026F00038344434443444343834003400340034FE
:102700007C34143414341434083400340034003469
:1027100008341434143418347C3400340034003455
:102720007C34083404340434083400340034003475
:102730004834543454345434203400340034003495
:1027400004343F3444344034203400340034003402
:102750003C344034403420347C3400340034003481
:102760001C342034403420341C3400340034003411
:102770003C344034303440343C3400340034003491
:1027800044342834103428344434003400340034C1
:102790000C345034503450343C3400340034003461
:1027A0004434643454344C344434003400340034FD
:1027B00000340834363441340034003400340034FA
:1027C000003400347F3400340034003400340034EA
:1027D00000344134363408340034003400340034DA
:1027E000043408340434083404340034003400342D
:1027F000003406340934093406340034003400341B
:102800000034003400340034003400340034003428
:102810000034003400340034003400340034003418
:102820000034003400340034003400340034003408
:1028300000340034003400340034003400340034F8
:102A100070345034703400340034003400340034E6
:102A2000003400340F3401340134003400340034F5
:102A3000013401340F3400340034003400340034E5
:102A40001034203440340034003400340034003476
:102A500000341834183400340034003400340034A6
:102A60000A340A344A342A341E3400340034003420
:102A700004344434343414340C340034003400341A
:102A800020341034783404340034003400340034FA
:102A9000183408344C3448343834003400340034AA
:102AA00048344834783448344834003400340034EE
:102AB0004834283418347C3408340034003400346A
:102AC00008347C340834283418340034003400349A
:102AD00040344834483478344034003400340034CE
:102AE0005434543454347C340034003400340034CE
:102AF000183400345834403438340034003400344E
:102B000008340834083408340834003400340034FD
:102B1000013441343D340934073400340034003486
:102B2000103408347C34023401340034003400346E
:102B30000E340234433422341E3400340034003462
:102B4000413441347F344134413400340034003462
:102B5000223412340A347F34023400340034003416
:102B600042343F34023442343E34003400340034C2
:102B70000A340A347F340A340A340034003400340E
:102B800008344634423422341E34003400340034D5
:102B90000434033442343E3402340034003400340C
:102BA00042344234423442347E34003400340034FF
:102BB00002344F3422341F340234003400340034E1
:102BC0004A344A34403420341E3400340034003453
:102BD0004234223412342A3446340034003400346F
:102BE00002343F3442344A34463400340034003432
:102BF00006344834403420341E3400340034003469
:102C0000083446344A3432341E340034003400343C
:102C10000A344A343E340934083400340034003471
:102C20000E3400344E3420341E340034003400346A
:102C3000043445343D340534043400340034003465
:102C400000347F340834103400340034003400344D
:102C5000443424341F340434043400340034003445
:102C6000403442344234423440340034003400347E
:102C700042342A3412342A34063400340034003406
:102C8000223412347B3416342234003400340034BD
:102C90000034403420341F34003400340034003415
:102CA000783400340234043478340034003400348E
:102CB0003F34443444344434443400340034003425
:102CC00002344234423422341E340034003400349E
:102CD0000434023404340834303400340034003412
:102CE000323402347F34023432340034003400345D
:102CF00002341234223452340E340034003400349E
:102D000000342A342A342A34403400340034003465
:102D10003834243422342034703400340034003405
:102D2000403428341034283406340034003400345D
:102D30000A343E344A344A344A34003400340034CD
:102D400004347F34043414340C340034003400343C
:102D50004034423442347E34403400340034003451
:102D60004A344A344A344A347E340034003400341D
:102D700004340534453425341C3400340034003424
:102D80000F34403420341F34003400340034003415
:102D90007C3400347E344034303400340034003429
:102DA0007E3440342034103408340034003400348D
:102DB0007E344234423442347E34003400340034B1
:102DC0000E340234423422341E34003400340034D1
:102DD0004234423440342034183400340034003457
:102DE000023404340134023400340034003400343A
:102DF0000734053407340034003400340034003420
:102E00000034003400340034003400340034003422
:102E10000034003400340034003400340034003412
:102E20000034003400340034003400340034003402
:102E300000340034003400340034003400340034F2
:102E400000340034003400340034003400340034E2
:102E500000340034003400340034003400340034D2
:102E600000340034003400340034003400340034C2
:102E700000340034003400340034003400340034B2
:102E800000340034003400340034003400340034A2
:102E90000034003400340034003400340034003492
:102EA0000034003400340034003400340034003482
:102EB0000034003400340034003400340034003472
:102EC0000034003400340034003400340034003462
:102ED0000034003400340034003400340034003452
:102EE0000034003400340034003400340034003442
:102EF0000034003400340034003400340034003432
:102F00000034003400340034003400340034003421
:102F10000034003400340034003400340034003411
:102F20000034003400340034003400340034003401
:102F300000340034003400340034003400340034F1
:102F400000340034003400340034003400340034E1
:102F500000340034003400340034003400340034D1
:102F600000340034003400340034003400340034C1
:102F700000340034003400340034003400340034B1
:102F800000340034003400340034003400340034A1
:102F90000034003400340034003400340034003491
:102FA0000034003400340034003400340034003481
:102FB0000034003400340034003400340034003471
:102FC0000034003400340034003400340034003461
:102FD0000034003400340034003400340034003451
:102FE0000034003400340034003400340034003441
:102FF0007F347F347F347F347F34003400340034B6
:02400E00323F3F
:00000001FF
